:100000000C9476000C94F40A0C9493000C949300D6
:100010000C9493000C9493000C9493000C94930014
:100020000C9493000C9493000C9493000C94930004
:100030000C9493000C9493000C9493000C949300F4
:100040000C9493000C9493000C9493000C949300E4
:100050000C9493000C9493000C9493000C949300D4
:100060000C9493000C9493000C9493000C949300C4
:100070000C9493000C9493000C94930009021200CA
:10008000010100806409040000000000000012016A
:100090001001FF000008C016DC050002010200018B
:1000A0001E0349004E004C00200052006500740001
:1000B00072006F002D00500072006F0067002A036D
:1000C00049006E00660069006E00690074006500FA
:1000D0004E00650073004C006900760065007300F7
:1000E0002E0063006F006D000403090411241FBE7D
:1000F000CFEFD4E0DEBFCDBF11E0A0E0B1E0E4E699
:10010000F8E102C005900D92A630B107D9F723E0BF
:10011000A6E0B1E001C01D92AA3AB207E1F70E9441
:10012000080C0C94300C0C9400000F931F93CF9389
:10013000DF93EC01FB01D9010091490110914A01C3
:10014000888187FF09C08E818C93442399F00481B4
:10015000158180E883831DC08FEF8C938E818093FF
:100160003401442309F44BC0709366036093650324
:1001700080E9F0CFE0912201F09123018381883D55
:10018000A1F50481158180E88383E0912201F0913B
:1001900023011782E0912201F091230183818039AC
:1001A000F1F48A81813711F08034C9F4E09165035C
:1001B000F09166030480F581E02D8C818083E091CD
:1001C0006503F09166030480F581E02D8D818183C4
:1001D000E0916503F091660387818E5F8783C80194
:1001E000DF91CF911F910F910895803D11F41C92E2
:1001F000CCCF8FEF8C9380E10E947B06C6CFE0913D
:100200002201F09123018381811106C0F0936603DE
:10021000E093650380E9B8CF883969F7E8CFE5E571
:10022000F1E08FEF819391E0E536F907D9F78093FC
:100230004801809327018093470180932601809392
:10024000380180931501809337018093140181E078
:100250000C947B06CF93DF93FC0150E0CA01820F20
:10026000911D4197E4F52223E1F183818F3FD9F578
:1002700082818F3FD1F5DA01AB5ABE4FED0180E0AC
:1002800099919F3FA1F58F5F2813FACF6283138264
:10029000982F9295990F907E915096831782108691
:1002A0001182108211861286138614861586168690
:1002B000178695E0440F551F9A95E1F720910001AC
:1002C00030910101420F531F5583448390E06D9399
:1002D0009F5F8913FCCF80E0DF91CF9108958EEB73
:1002E000FBCF82ECF9CF8FEBF7CF80ECF5CF81EC31
:1002F000F3CFCF93DF93DC01EB019A0112969C912F
:10030000129780ED890F803318F513968C9113970F
:10031000813041F0E8F08230A9F08330B1F085EB14
:10032000888346C0E4E2F1E0913509F476C048F5EF
:10033000913309F449C078F49923B9F19033E1F18C
:1003400084EBEECFE5E3F1E0EFCFE2E1F1E0ECCFDB
:10035000E5E4F1E0E9CF933309F446C0E8F19035E4
:1003600079F7188286E0898386818A8383818B83EB
:1003700087818C8380858D8382818E8387858F831F
:1003800017C0903808F05FC0903708F055C090361D
:1003900079F19136C9F1923599F6188282E0898314
:1003A00080818A8381818B8303C00E940F01188220
:1003B000CE01DF91CF91089514968C9114971596E4
:1003C0009C9191878287F3CF14968C911497159600
:1003D0009C9193878487EBCF14968C9114971596F4
:1003E0009C9195878687E3CF14968C918787DFCF82
:1003F000188281E089831496ED91FC911597EB5A50
:10040000FE4F80818A83D4CF188281E08983E09176
:100410002201F09123018381F5CF188286E0898340
:1004200081858A8382858B8383858C8384858D8374
:1004300085858E838685A3CF40E0BF01CD01DF9106
:10044000CF910C949500892F8770813049F0F8F096
:10045000823001F1833009F062CFE2E1F1E002C0C5
:10046000E4E2F1E0903808F4A3CF9838B0F0905966
:10047000983008F09DCF188213968C91139780873F
:1004800014968D919C9115979183808391CFE5E48B
:10049000F1E0E8CFE5E3F1E0E5CF14964C91149755
:1004A00015966C91159713962C91CF010E942A01F5
:1004B00037CF90914801809127018F3F79F481E0F7
:1004C0009F3F09F480E0909138019F3F09F083E05D
:1004D000909115019F3F09F084E0089582E0F3CFE9
:1004E000623059F421E08534920749F121E08432E9
:1004F000920789F485E491E00EC0633069F421E04D
:1005000085349207E1F021E084329207D9F021E0AE
:100510008533920779F308956430E9F721E0853453
:10052000920769F021E08432920761F021E085337F
:10053000920759F021E08231920769F7DBCF84E21C
:1005400091E0089585E391E0089582E191E00895B6
:100550001F93CF93DF930E948106823D09F071C003
:100560000E9459028093060185E491E09093230153
:10057000809322010E948106823DA1F4D091060160
:100580008091220190912301C1E0CD1708F45FC052
:10059000909323018093220120E8FC01238380EDC6
:1005A0000E947B060E948106823F41F480EF0E94F8
:1005B0007B06E0912201F091230113820E948106C3
:1005C000C82F803DE1F48091220190912301FC012C
:1005D00023812038A1F4609106010E94700290935B
:1005E000230180932201FC011782C3830E944003F0
:1005F000E0912201F0912301882371F183830E940D
:100600008106182F803FC9F4C0912201D0912301A7
:100610008B81883991F460910601CE010E947002AD
:100620009093230180932201FC0113821B83CE014E
:100630000E9422048823D1F08B83DF91CF911F91F8
:1006400008950E948106823F09F094CF89CF6D2FD3
:100650000E947002CF5F99CF88ED838320858081CF
:100660009181820F911D91838083C9CF84EF8B8309
:10067000288588819981820F911D99838883DDCF98
:100680000F93CF93DF93EC0168818985823101F16B
:1006900030F4803159F0813191F083EC03C0853121
:1006A000E0F780E0DF91CF910F91089560680FEF40
:1006B0002E814A818C819D810E94EA0507C00FEF3F
:1006C0002E814A818C819D810E9422068F83E9CFF1
:1006D0006066EDCF7F928F929F92AF92BF92CF9242
:1006E000DF92EF92FF920F931F93CF93DF936A01F4
:1006F0005901DA011796CC91D0E0E62EF12CFE2CB0
:10070000EE24D60116968C91169790E08C179D07D3
:1007100088F41796CC9380E0DF91CF911F910F91D1
:10072000FF90EF90DF90CF90BF90AF909F908F9011
:100730007F9008956AEA85E595E5F501099565E5F7
:100740008AEA9AE2F501099560EA85E595E5F50101
:100750000995CE0199274C018E289F28D601149621
:10076000ED91FC911597E80FF91F6081C401F50127
:1007700009950E94D509C401F8010995782EC40194
:10078000F80109957812F5CF2196BBCF7F928F9211
:100790009F92AF92BF92CF92DF92EF92FF920F9310
:1007A0001F93CF93DF936A015901DA011796CC9119
:1007B000D0E0E62EF12CFE2CEE24D60116968C917C
:1007C000169790E08C179D0788F41796CC9380E0DD
:1007D000DF91CF911F910F91FF90EF90DF90CF901D
:1007E000BF90AF909F908F907F9008956AEA85E5C3
:1007F00095E1F501099565E58AEA9AE0F501099523
:1008000060EA85E595E1F5010995CE0199274C014E
:100810008E289F28D6011496ED91FC911597E80F2C
:10082000F91F6081C401F50109950E94D509C40131
:10083000F8010995782EC401F80109957812F5CFD1
:100840002196BBCF0F931F93AC01FC016081818582
:100850008131A1F020F4803141F083EC03C0853177
:10086000E0F780E01F910F91089560680EEF14E0AB
:1008700023EE34E080E00E946A03F3CF0CE315E03E
:1008800020E535E080E00E94C603EBCF3F9A479811
:100890008FEF81B911B882B914B885B914B885B988
:1008A0003898409A3998419A3A98429A3C98449A92
:1008B0003D98459A3E98469A53985B9A55985D9A0A
:1008C0003F98479A57985F9A3B98439A5098589800
:1008D0005198599A08950E944604399A419A389A33
:1008E00040983A9A429A3C9A449A3D9A459A14B84A
:1008F0008FEF85B914B885B93F9A479881B912B876
:1009000084B915B80E94980614B808955898509A5A
:10091000000089B15098589880FD22C05098589A8C
:1009200059B149B1000039B10000000029B10000FF
:100930000000000099B1000000000000000089B133
:100940005098589850FD0EC040FD0EC030FD0EC0AE
:1009500020FD0EC090FD0EC080FD0EC080EE0895FB
:1009600080EF089580E0089581E0089583E0089580
:1009700086E008958AE008958FE008950F931F930D
:10098000CF93DF931F92CDB7DEB78901813079F025
:1009900020F0803881F086E904C089830E944604F3
:1009A00089810F90DF91CF911F910F9108950E943F
:1009B0006B0480E0F6CF81E0F90180830E94860419
:1009C000F8018183F6CF1F93CF93DF931F92CDB7AA
:1009D000DEB782B91FEF14B995B969830E949806F2
:1009E00014B814B9698165B9509A58985098589AB2
:1009F00014B80F90DF91CF911F910895CF93DF939B
:100A0000EC0182B98FEF84B9D5B90E94980614B869
:100A1000409AD7FD4198000000000000000083B11B
:100A20004098419ADF91CF910895EF92FF921F93E2
:100A3000CF93DF931F92CDB7DEB77C0150985898C3
:100A400082B91FEF14B9F5B869830E94980614B8EB
:100A5000429814B9698165B9409AF7FC4198000041
:100A600000004098419A429A14B80F90DF91CF91BC
:100A70001F91FF90EF900895811520E2920708F4EE
:100A8000906882B98FEF84B995B90E94980614B81E
:100A90004498000000000000000083B1449A0895CB
:100AA0001F93CF93DF931F92CDB7DEB7811520E25E
:100AB000920708F4906882B91FEF14B995B9698359
:100AC0000E94980614B814B9698165B90000459868
:100AD0000000459A14B80F90DF91CF911F910895AF
:100AE0001F93CF93DF931FEF14B984E085B90E9461
:100AF000980614B8C9B1C072D0E014B988E085B9BD
:100B00000E94980614B889B1807290E031E0209775
:100B100009F030E051E0009709F050E0332311F084
:100B2000511119C041E0CD2B09F440E021E0892B9F
:100B300009F420E0442311F021110FC0552311F0D6
:100B400041110DC0332311F021110BC08FEFDF9144
:100B5000CF911F91089580E1FACF81E1F8CF82E132
:100B6000F6CF83E1F4CF0F931F93CF93C82FCA0121
:100B70008901C23001F130F4CC2391F0C130B9F0D9
:100B8000C0EA10C0C238D1F0C338F1F0C138C1F7A3
:100B900021E0F80120830E94FE04F801818309C04E
:100BA0000E94E3048C2FCF911F910F9108950E9412
:100BB0005005C0E0F7CF0E941505FBCF21E0F801FA
:100BC00020830E943C05E9CF81E0F90180830E94E7
:100BD0007005E3CFDF92EF92FF920F931F93CF93B5
:100BE000DF931F92CDB7DEB77C01142FD22E8FEF8B
:100BF00084B965B969830E94980614B8409A6981DE
:100C000067FD419812B980E0011117C00000000093
:100C100093B1F701E80FF11D90831F5F12B98F5F49
:100C2000D81690F74098419A0F90DF91CF911F917D
:100C30000F91FF90EF90DF90089589830E94D5096E
:100C40008981E6CFDF92EF92FF920F931F93CF93AC
:100C5000DF931F92CDB7DEB77C01142FD22E603206
:100C600008F460688FEF84B965B90E94980614B8DB
:100C7000449812B980E0011116C00000000093B141
:100C8000F701E80FF11D90831F5F12B98F5FD8162F
:100C900090F7449A0F90DF91CF911F910F91FF90A1
:100CA000EF90DF90089589830E94D5098981E7CF6D
:100CB000CF93DF93FB01DC0112962C91222329F0C4
:100CC000203479F082ED808308C01082A091020167
:100CD000B0910301EC018C818C93CF01DF91CF9116
:100CE0000895108281E08183A0910201B0910301F7
:100CF0008C918283F2CFE0910201F0910301808315
:100D00000895E0910201F09103018081089585B179
:100D10008093070192B12091080125B92FEF21B9E5
:100D200082B93F9A4798479A479885B992B90895EA
:100D300085B18093080182B19FEF91B9909107012D
:100D400092B9479A479882B908950F931F93D90192
:100D5000082F10E00531110508F09BC2F801ED5491
:100D6000F94F0C942A0CEA06C80623077C07C6072D
:100D700010085A08FC080109060909090D0910099B
:100D800018091E0922092509290932093B094109C7
:100D90004631510508F07FC2FA01EF52F94F0C9429
:100DA0002A0CE706ED06F1064B09F506F906FD06E5
:100DB0000107050709070D071107150719074B0953
:100DC0004B094B094B094B094B094B091F07389835
:100DD000409A80E01F910F9108953998419A80E0E0
:100DE000F9CF3A98429A80E0F5CF3C98449A80E057
:100DF000F1CF3D98459A80E0EDCF3E98469A80E04D
:100E0000E9CF3F98479A80E0E5CF5098589A80E024
:100E1000E1CF5198599A80E0DDCF53985B9A80E0FA
:100E2000D9CF55985D9A80E0D5CF56985E9A80E0EC
:100E3000D1CF57985F9A3B98439A80E0CBCF509898
:100E4000589A80E0C7CF4631510508F026C2FA0112
:100E5000E45DF84F0C942A0C420746074A074D09F7
:100E60004E07520756075A075E07620766076A076A
:100E70006E0772074D094D094D094D094D094D0980
:100E80004D0978073898409880E0A4CF3998419868
:100E900080E0A0CF3A98429880E09CCF3C9844985C
:100EA00080E098CF3D98459880E094CF3E98469852
:100EB00080E090CF3F98479880E08CCF509858982A
:100EC00080E088CF5198599880E084CF53985B9800
:100ED00080E080CF55985D9880E07CCF56985E98F2
:100EE00080E078CF57985F983B98439880E072CF26
:100EF0005098589880E06ECF4631510508F0CFC128
:100F0000FA01EB57F84F0C942A0C9B079E07A10798
:100F10004F09A407A707AA07AD07B007B307B6078D
:100F2000B907BC07BF074F094F094F094F094F09C0
:100F30004F094F09C307389A80E04CCF399A80E0B7
:100F400049CF3A9A80E046CF3C9A80E043CF3D9A21
:100F500080E040CF3E9A80E03DCF3F9A80E03ACF9C
:100F6000509A80E037CF519A80E034CF539A80E096
:100F700031CF559A80E02ECF569A80E02BCF579AEA
:100F80003B9A80E027CF509A80E024CF463151052C
:100F900008F087C1FA01E153F84F0C942A0CE507D9
:100FA000E807EB075109EE07F107F407F707FA071F
:100FB000FD070008030806080908510951095109ED
:100FC00051095109510951090D08409880E002CF9B
:100FD000419880E0FFCE429880E0FCCE449880E0CB
:100FE000F9CE459880E0F6CE469880E0F3CE47985B
:100FF00080E0F0CE589880E0EDCE599880E0EACEBF
:101000005B9880E0E7CE5D9880E0E4CE5E9880E07B
:10101000E1CE5F98439880E0DDCE589880E0DACE4C
:101020004631510508F03FC1FA01E75EF74F0C94D5
:101030002A0C2F0832083508530938083B083E08A7
:101040004108440847084A084D0850085308530906
:101050005309530953095309530953095708409A2F
:1010600080E0B8CE419A80E0B5CE429A80E0B2CE20
:10107000449A80E0AFCE459A80E0ACCE469A80E0BC
:10108000A9CE479A80E0A6CE589A80E0A3CE599A7E
:1010900080E0A0CE5B9A80E09DCE5D9A80E09ACE03
:1010A0005E9A80E097CE5F9A439A80E093CE589AFA
:1010B00080E090CE82E08C934631510508F099C0D3
:1010C000FA01EB59F74F0C942A0C7B0884088D0821
:1010D000F90896089F08A808B108BA08C308CC0800
:1010E000D508DE08E708F908F908F908F908F90849
:1010F000F908F908F00886B1817011968C93119760
:1011000012961C9280E066CE86B1827090E01296B4
:101110009C938E93119780E05DCE86B1847090E0B1
:1011200012969C938E93119780E054CE86B1807175
:1011300090E012969C938E93119780E04BCE86B1EF
:10114000807290E012969C938E93119780E042CE2D
:1011500086B1807490E012969C938E93119780E0F4
:1011600039CE86B1807890E012969C938E93119739
:1011700080E030CE89B1817011968C9311971296D0
:101180001C9280E027CE89B1827090E012969C93E9
:101190008E93119780E01ECE89B1887090E01296F0
:1011A0009C938E93119780E015CE89B1807290E068
:1011B00012969C938E93119780E00CCE89B1807427
:1011C00090E012969C938E93119780E003CE89B1A4
:1011D000807890E012969C938E93119780E0FACDE0
:1011E00089B1817011968C93119712961C9280E0B0
:1011F000F1CD1C928DE8EECD14B88FEF85B980E06B
:10120000E9CD14B88FEF85B980E0E4CD14B880E063
:10121000E1CD8FEF84B980E0DDCD45B980E0DACD56
:1012200083B111968C93119781E08C9380E0D2CD9D
:101230003F9A47988FEF81B980E0CCCD8FEF82B98C
:1012400080E0C8CD11B880E0C5CD8FEF81B980E0D6
:10125000C1CD42B98FEF84B955B90E94980614B830
:1012600080E0B8CD14B88FEF85B9579A5F983B9A54
:10127000439880E0AFCD57985F9A3B98439A80E0BF
:10128000A9CD8FEF84B945B90E94870614B880E0D4
:10129000A1CD8CE89FCD8DE89DCD8DE89BCD8DE8CF
:1012A00099CD8DE897CD8DE895CDCF93DF931F92A3
:1012B000CDB7DEB7FC018FEF8093090110920A01D0
:1012C00089E091E090938F0380938E0386818983D8
:1012D0008181833041F130F4813089F08230D1F066
:1012E00080E815C0853041F18730D1F7AE014F5FFE
:1012F0005F4F69E071E0CF010E94580625C044812C
:1013000055812AE031E0638182810E94A5068093A5
:1013100009011EC0448155812AE031E06381828148
:101320000E94BE04F4CF448155812AE031E06381FC
:1013300082810E94B305EBCFAE014F5F5F4F69E042
:1013400071E0CF010E94790190938F0380938E0307
:1013500089810F90DF91CF910895E0916503F0911D
:101360006603278144815581322F360F231312C023
:10137000E0916503F09166038781860F87838091F2
:101380003401861B8093340181110DC088E9838369
:1013900081E00895FC017191CF01FA01E20FF11D86
:1013A00070832F5FE3CF80E00895CF93DF93609148
:1013B0009003635067FD91C080918D03CCE0D0E035
:1013C000C81BD109CC56DC4F80918C038D3209F0BB
:1013D000CFC0683009F07FC083EC809380038AE53A
:1013E00080930501109211018881807679F0CE01F9
:1013F0000E9455098F3F09F466C09F81911169C011
:101400009E81981708F065C0892F63C02A811092C9
:101410008903998191110AC010928A0329E833E067
:1014200082E030938F0320938E03E7CF953029F429
:101430002093910329E833E0F4CF963099F59B810E
:10144000913059F48EE890E090938F0380938E034F
:1014500082E190E490931101D0CF923019F48CE79F
:1014600090E0F2CF9330A9F7211108C088EE90E008
:1014700090938F0380938E0384E0EBCF213041F46F
:101480008EEB90E090938F0380938E038AE2E1CFFE
:101490002230F9F680EA90E090938F0380938E03D8
:1014A0008EE1D7CF983059F0993019F420939303F7
:1014B000C1CF81E09A3009F4BDCF80E0BBCF23E9F2
:1014C00033E081E0AECF988197FD8E8190E89093D4
:1014D000110180930401109290038091050184FF13
:1014E0003AC0809104018F3FB1F1C82F893008F0D4
:1014F000C8E08C1B809304018091800398E88927C1
:1015000080938003CC23D1F080918E0390918F0340
:101510002091110126FF3FC0A1E8B3E0FC012C2F70
:1015200034913D9331962150D9F701962FEF2C0F2E
:10153000820F911D90938F0380938E036C2F81E80F
:1015400093E00E94F00ACC5FCC3019F08FEF8093CB
:101550000401C093050184E199B1947131F4815083
:10156000D9F71092910310928B03DF91CF910895D8
:101570008091110187FFAFCFCE010E94AD098F3F4F
:1015800021F48EE180930501A6CF882309F4A3CF2F
:1015900010920401A0CFE1E8F3E0DC012C2F3D9193
:1015A00031932150E1F7C1CFE9E6F0E0808182601C
:1015B0008083E89A0895A82FB92F80E090E041E059
:1015C00050EA609530E009C02D9182279795879564
:1015D00010F084279527305EC8F36F5FA8F3089555
:1015E000EADF8D939D930895CF93CFB7CF93DF9389
:1015F000C3954C9BE9F74C9B0BC04C9B09C04C9B83
:1016000007C04C9B05C04C9B03C04C9B01C089C0CC
:101610006F93C0918D03DD27CC56DC4F2F9365E58A
:101620004C9B03C02F916F91E6CF0F931F934F9365
:1016300020E040E15F9309B1047104FB27F93F9377
:1016400050E03BE039C0147140642F77012F5F5F99
:101650001EC0406819B114712F7752501FC04064EA
:1016600009B12F770471D1F15F5F00C023C04062E0
:1016700019B12F77147191F15F5F00C025C004711B
:101680001027515012F45D5F0000115027952C3F38
:1016900019B1C8F614710127015027952C3FC8F6DF
:1016A0004227499309B1047110274F7311502795B0
:1016B0002C3FA8F64695469519B1147179F001278B
:1016C000015027952C3F98F66B5A60F3315009B1C1
:1016D000B0F600C011E01CBB002717C03B5031958D
:1016E000C31BD04011E01CBB0881033CF9F00B3454
:1016F000E9F020918B031981110F1213EDCF0936F8
:1017000051F10D3211F0013E39F7009392033F91F0
:101710005F914F911F910F912F916F91CCB3C0FDAD
:1017200067CFDF91CF91CFBFCF91189520919203D2
:10173000222369F310919003112339F534303AF1E3
:101740003093900320938C0310918D033BE0311B69
:1017500030938D031CC0009190030130B4F40AE56E
:101760003091050134FD14C000930501C0E8D3E0B9
:1017700013C0052710E000C000000BB91AC00527F0
:1017800010E0221F1DC010E021C04AE502C032ED6A
:10179000432FC4E1D0E032E01AB114615C9A0BB17E
:1017A0001AB954E120E865E320FF05270BB9279516
:1017B00017951C3FF0F66695B8F7B1F720FF05279F
:1017C0000BB9279517951C3FD0F62795179517FF4E
:1017D000052700001C3F0BB9B0F629913A9519F77F
:1017E0000B7E10919103110FC651D0400BB911F02F
:1017F00010938B0311E01CBB00611AB11B7E402FBC
:101800004B7E54E05A95F1F70BB91AB94BB97FCF1B
:101810009EE088E10FB6F894A895809360000FBE13
:10182000909360000E94D40A549A80E0815051F451
:10183000549878940E944604A8950E94D5090E9465
:10184000A802FACFA895EFE9FFE03197F1F700C0C1
:101850000000ECCFEE0FFF1F0590F491E02D0994EE
:04186000F894FFCF2A
:0618640065016703FF5A55
:00000001FF
